:020000040801F1
:10C800001C491B4808601D491B4808601D491C48FD
:10C8100008601E491C4808601E491D4808601F49E1
:10C820001D4808601F491E48086020491E480860CE
:10C8300020491F48086021491F48086021492048B5
:10C84000086022492048086022492148086023499D
:10C85000214808602349224808602449224808608A
:10C860002449234808602549234808607047000090
:10C87000FBD301083C070020C7CA0108400700207D
:10C880006BCA0108F4050020E5C90108F80500207D
:10C89000E3C90108FC05002065C901080006002065
:10C8A00063C901080406002061C9010808060020C8
:10C8B0005FC90108100600205DC9010814060020A8
:10C8C0005BC901084407002055C901080C06002077
:10C8D00053C901081806002051C901084807002063
:10C8E0004FC901081C060020452C00082006002026
:10C8F00001C90108240600207B0800203807002019
:10C90000FD4810B500780022FC49012808D0FC48F9
:10C91000007888B1012811D0022811D0032811D045
:10C920000A70F94AF74C0978126820789047207805
:10C9300058B10020207010BD0C2004E00E2002E051
:10C94000112000E012200870EBE70120F2E77047A9
:10C9500070477047ED480068004770477047704760
:10C96000704770472DE9F041E74C0C210120226807
:10C9700090470E2122680120904711212268012052
:10C9800090471221226801209047E148E14DE24E94
:10C99000006828600621326800209047DF4F286831
:10C9A000396888470721326800209047396828682D
:10C9B0008847DB4901200870226817219047D94831
:10C9C000007800280BD00420E6F7EBFCCC49087077
:10C9D000D649D54809688847D54900200870BDE880
:10C9E000F0817047D3490020D34A0870487088709E
:10C9F000C870087148718871C871087210704872E7
:10CA00008872C872087348738873C873087448744E
:10CA10008874C874087548758875C875087648762E
:10CA20008876C876087748778877C449C44A0870FA
:10CA300001211170C34A1070C34A1060B84A1170C6
:10CA4000C24A1170C24A1070C24A1060C24A1170C4
:10CA5000C2490860C2490870C2490860C2490870EA
:10CA6000C2490870C24908707047C2490020C24AD2
:10CA7000087001211170C14A1070C14A1070C14A7A
:10CA80001070C14A1060C14A1070C14A1060C14A9A
:10CA90001060C14A1070C14A1060C14A1060C14A9A
:10CAA0001070C14A1060C14A1060C14A1070C14A7A
:10CAB0001060C14A1170C24AC0491160C149087072
:10CAC000C14908607047C14910B50A200870C049C3
:10CAD00014208D4C0870BF4917200870BE490020F3
:10CAE000087048708870C8700871BC490870BC49EB
:10CAF00008700C2122680120904711212268012032
:10CB0000904712212268012090470E2122680120BF
:10CB10009047B4490E20087010BD8648417B00291B
:10CB200009D0807D002806D08449774A012008700A
:10CB300012680921104770472DE9F0417D4904230F
:10CB400008468F79704D00780226804C0322FFB191
:10CB50000F7AAFB190B18F7887B1C87958B1487862
:10CB600048B1C87838B1087928B10B212A6801206A
:10CB700090470A2000E00520207023E0CF799FB97C
:10CB8000CF7817B108B1227003E08F7807B1267013
:10CB900030B1487808B1887830B9087A00B1267089
:10CBA000C87818B1087908B123700BE0487810B143
:10CBB000C87900B12270887820B1087910B1087A5C
:10CBC00000B122705349C820086054490968884759
:10CBD0000D212A680020904710212A6800209047E4
:10CBE0002A68BDE8F0410F210020104770B57E4C47
:10CBF0004FF47A763046216888474E4D287810B138
:10CC0000216830468847687810B1216830468847E7
:10CC1000A87810B1216830468847E87810B12168BB
:10CC200030468847287910B1216830468847A8796E
:10CC300010B1216830468847E87910B12168304644
:10CC40008847287A002804D030462168BDE8704023
:10CC5000084770BD70B5324D5D4C28782178884208
:10CC60000DD262480068804728782178884206D132
:10CC7000254A212101201268BDE87040104770BD8F
:10CC800070B55B494FF47A70086057490968884766
:10CC9000FFF7E0FF274C607908B1FFF7A7FFE07BC3
:10CCA000002827D0207C002824D0607C002821D0B8
:10CCB000A07C00281ED0E07C00281BD001206073DF
:10CCC000114D207020722A680A21904722212A687B
:10CCD00001209047FFF730FFFFF71FFF0020E073B0
:10CCE000207460740C4AA074E0741268BDE870404F
:10CCF000062110477EE000009505002082050020F7
:10CD00009605002093050020A8040020EC040020D4
:10CD1000340400209C0500209C040020E404002032
:10CD200065050020CE030020D4060020C0040020AA
:10CD3000940500205C0800202A0700202F0700200F
:10CD4000630500206405002098050020660500208A
:10CD5000670500202007002028070020A0050020EC
:10CD6000290700201C070020680500206905002015
:10CD70006A0500206B0500206C0500206E05002070
:10CD80006F05002070050020B00500202B07002053
:10CD9000B4050020B80500202C070020BC050020A9
:10CDA000C00500202D070020C4050020C805002074
:10CDB0002E070020CC0500207105002040420F0006
:10CDC000D0050020720500202407002088050020DF
:10CDD00083050020600500202C0600207D05002032
:10CDE0007E05002024040020D4040020C804002074
:10CDF000D405002070BDFD48C17C002902D101216D
:10CE0000C1743DE77047F948817C002902D10121B6
:10CE1000817435E77047F548417C002902D1012132
:10CE200041742DE77047F148017C002902D10121AE
:10CE3000017425E77047ED48C17B002902D101212B
:10CE4000C1731DE7704770B5E9494FF47A70086007
:10CE5000E84909688847FFF7FDFEE44CE07A08B12D
:10CE6000FFF7C4FE207E002827D0607E002824D053
:10CE7000A07E002821D0E07E00281ED0207F002840
:10CE80001BD00120A075DC4DA071A0702A68242160
:10CE9000904707212A6801209047FFF74DFEFFF7D2
:10CEA0003CFE002020766076A076D44AE07620779B
:10CEB0001268BDE870400721104770BDCB48017F64
:10CEC000002902D101210177BDE77047C748C17E23
:10CED000002902D10121C176B5E77047C348817EA0
:10CEE000002902D101218176ADE77047BF48417E1C
:10CEF000002902D101214176A5E77047BB48017E98
:10CF0000002902D1012101769DE77047B94910B58A
:10CF1000096840F6B8308847BDE810400CE610B507
:10CF2000B249B54C012088712268242190470D2117
:10CF3000226801209047BDE81040E7E710B5AB49F3
:10CF4000AD4C0120C8712268232190470D21226831
:10CF500001209047BDE81040D8E710B5A349A64C82
:10CF6000012008722268222190470D2122680120A9
:10CF70009047BDE81040C9E79D4910B532200860D0
:10CF80009C49096888479E480078052813D397482C
:10CF9000C17A00290FD0817F00290CD1817A09B193
:10CFA000002100E001218172934A142102201268BD
:10CFB000BDE81040104710BD10B58C498E4C0120C3
:10CFC000C8702268052190470F21226801209047F0
:10CFD000BDE810409AE7884A10B50F211268012079
:10CFE0009047BDE8104091E710B58049824C012080
:10CFF00008712268062190470F212268012090477E
:10D00000BDE8104082E77A4910B5322008607949BE
:10D01000096888477A480078052813D3734841790E
:10D0200000290FD0817F00290CD1417A09B100215C
:10D0300000E001214172704A132102201268BDE80C
:10D040001040104710BD10B568496B4C01200870A6
:10D0500022680A2190471021226801209047BDE8EC
:10D06000104053E710B56149634C012048702268B5
:10D07000082190471021226801209047BDE8104008
:10D0800044E710B559495C4C01208870226807219B
:10D0900090471021226801209047BDE8104035E7F5
:10D0A00053490A20086053490968084710B5FFF73B
:10D0B000D1FD524A082100201268BDE810401047F7
:10D0C00010B54D4C1321002022689047142122688E
:10D0D000002090474B480068804744480021417237
:10D0E00081720121817710BD404810B5807A08B166
:10D0F000FFF7E6FF3E4940F6B83008603D49096851
:10D100008847BDE81040D1E770B5384CE07A002878
:10D1100013D1607F002810D0207D00280DD001267B
:10D12000354DE67216212A6830469047A6722A6865
:10D13000BDE8704014210120104770BD70B52B4D23
:10D140002B4C2C4E687F28B14FF4FA702060316868
:10D15000884719E0284A0C210020126890472A4885
:10D16000007840B12948007828B92948007810B9DA
:10D1700028480068804741F288302060316888473D
:10D1800001206877FFF7C0FFBDE870408EE72DE90A
:10D19000F05F214DDFF884904FF47A782878204EA4
:10D1A0000A38C7B2DFF87CA0DFF87CB018E099F845
:10D1B0000040E9F7CEFF07E04046EAF732F9306871
:10D1C000ECF77CFF641EE4B2002CF5D1DAF8000025
:10D1D00080472878401E2870DBF80000ECF76EFFCF
:10D1E0002878B842E3D8BDE8F09F00005C08002032
:10D1F000D4050020D4040020A80400209C040020B2
:10D20000BB0300205C040020CE0300206B0500203F
:10D2100096050020D8040020650500206605002042
:10D2200028040020980400203004002070B5CC4D64
:10D2300028780A280BD3CB4C212100202268904764
:10D24000FFF7A5FF01202870226817219047C649E3
:10D250004FF47A7009688847BDE8704026E770B5DA
:10D26000C24CC34DC04E207D28B14FF4FA702860E7
:10D27000316888471AE0BB4A0E21002012689047A7
:10D28000BC48007848B1BC48007830B9BB48007849
:10D29000012802D1BA48006880470120207541F278
:10D2A0008830286031688847FFF72EFFBDE870405E
:10D2B000FCE6AE4810B5407A08B1FFF701FFAC4973
:10D2C00040F6B8300860A84909688847BDE81040B2
:10D2D000ECE670B5A54C6079002813D1E07D0028FC
:10D2E00010D0A07B00280DD001269E4D667115211F
:10D2F0002A683046904766722A68BDE8704013215C
:10D300000120104770BD70B5984D994C964EE87D40
:10D3100028B14FF4FA702060316888471AE0914ACA
:10D3200011210020126890479248007848B1924835
:10D33000007830B991480078022802D190480068FE
:10D34000804741F288302060316888470120E875C5
:10D35000FFF7BFFFBDE87040A8E610B5894C207804
:10D3600068B1894800688047002020708748884954
:10D370007C4A007808600921126800209047FFF776
:10D38000C5FD84480068BDE8104000478248784ADF
:10D3900003787548052B016802D24FF47A7000E0DB
:10D3A00064201060084770B5704D714C6E4EA87BBC
:10D3B00028B14FF4FA702060316888471AE0694A52
:10D3C00012210020126890476A48007848B16A48E4
:10D3D000007830B969480078032802D168480068AD
:10D3E000804741F288302060316888470120A87367
:10D3F000FFF76FFFBDE8704058E610B52A286CD0E3
:10D400001FDC172851D00BDCA0F10A000C2870D2C9
:10D41000DFE800F036393C3F4295959595954548B3
:10D4200020284ED006DC182842D01E2843D01F28C2
:10D430005FD143E0222847D0282848D029287ED130
:10D4400048E03E2862D010DC342853D006DC2C287B
:10D4500046D0322847D0332871D147E036284CD007
:10D460003C284DD03D286AD14DE03F380C2866D28B
:10D47000DFE800F04F52656565656555585B5E6194
:10D48000FFF791FF59E0FFF781FF56E0FFF765FFD7
:10D4900053E0FFF738FF50E0FFF70BFF4DE0FFF7D9
:10D4A000DEFE4AE0FFF7C2FE47E0FFF747FE44E03A
:10D4B000FFF71AFE41E0FFF7F3FD3EE0FFF7E1FD65
:10D4C0003BE0FFF7CFFD38E0FFF7BDFD35E0FFF7AC
:10D4D0009AFD32E0FFF788FD2FE0FFF77CFD2CE09E
:10D4E000FFF76AFD29E0FFF747FD26E0FFF735FD6E
:10D4F00023E024E0FFF722FD1FE0FFF710FD1CE012
:10D50000FFF7FCFC19E0FFF7F1FC16E0FFF7E6FC83
:10D5100013E0FFF7DBFC10E0FFF7D0FC0DE0FFF7B6
:10D520008AFC0AE0FFF77FFC07E0FFF774FC04E0E9
:10D53000FFF769FC01E0FFF75EFC002010BD4FF033
:10D54000FF3010BD70471448094A03780648032B82
:10D55000016802D06420106008474FF47A70FAE73F
:10D5600065050020A8040020D40400205C080020E9
:10D57000D4050020CE0300206B0500209605002076
:10D58000D80400202F070020800400206C05002014
:0CD59000A0050020C8040020BB03002000
